:10000000AEC014C2C6C0C5C0C4C0C3C0C2C0C1C097
:10001000C0C0BFC0BEC0BDC0BCC0BBC0BAC0B9C0FC
:10002000B8C0B7C0B6C00403090418037200610069
:10003000700068006E00650074002E006E006500A0
:10004000740022032800530029004E00450053008D
:100050002F00410074006100720069005F005500CC
:10006000530042000A033100300030003000050127
:100070000905A1010901A10009300931150026FF78
:1000800000750895028102C00509190129081500AB
:100090002501750195088102C005010902A1010928
:1000A00001A1000509190129021500250195027514
:1000B0000181029501750681030501093009311599
:1000C00081257F750895028106C0C01201010100DB
:1000D0000000088117970A060101020001050109C5
:1000E00005A1010901A10009300931150026FF0011
:1000F000750895028102C00509190129041500251A
:1001000001750195048102750195048103C01201F6
:100110000101000000088117990A0601010200018F
:1001200005010905A1010901A100093009311500E6
:1001300026FF00750895028102C0050919012908EA
:1001400015002501750195088102C0120101010009
:100150000000088117960A0601000003010011241F
:100160001FBECFE5D4E0DEBFCDBF10E0A0E6B0E01B
:10017000E8E8F3E102C005900D92A43DB107D9F77C
:1001800011E0A4EDB0E001C01D92A733B107E1F783
:1001900036C336CF85B7836085BF8BB780648BBF8E
:1001A00083EC80930D0108950F931F93CF93DF93FA
:1001B00090911D0119160CF0A6C020911A01809192
:1001C00019018D3209F097C08AE5809361009B3058
:1001D00009F091C0CDE2D1E0C21BD10988818076BF
:1001E00009F07BC02BE031E010920B01898188235C
:1001F00041F410920C0130931C0120931B0192E0FA
:1002000006C0853031F48A8180931E0190E020E899
:100210006AC0863009F043C08B818130E1F18230C1
:1002200019F4CE0166D25BC0833049F58A818823F8
:1002300041F486E290E090931C0180931B0194E0CE
:1002400051C0813041F48AE290E090931C01809388
:100250001B0198E147C0823041F482E490E0909322
:100260001C0180931B0192E23DC08330D1F584E6EE
:1002700090E090931C0180931B019CE033C081327D
:1002800041F487EE90E090931C0180931B0199E06C
:1002900029C0823231F5CE012CD2982F23C088306C
:1002A00039F480E291E090931C0180931B010CC013
:1002B000893021F48A8180932001A8CF8A3031F4DB
:1002C00030931C0120931B0191E0A1CF8B3009F0EA
:1002D0009DCF83EC80930D0199CFCE013BD2982F17
:1002E00096CF90E020EC8F81882339F48E81891796
:1002F00020F4982F02C090E020E82093D40090933F
:10030000600010921D018091610084FF41C08091C6
:1003100060008F3F09F43CC0682F893008F068E026
:10032000861B809360008091D40080FF02C003ECA4
:1003300001C00BE48F5F8093D400E0911B01F0912A
:100340001C0186FD04C0962FA3E0B1E00CC0962FDF
:10035000A3E0B1E003C084918D9331969150D8F71A
:1003600004C081918D939150E0F7F0931C01E093CC
:100370001B017727162F83E091E054D0183018F432
:100380008FEF80936000009302011C5F1093610067
:100390009AE080B3857031F49150D9F710921E0124
:1003A00010921801DF91CF911F910F9108951F9323
:1003B000DC01162F8091620084FF07C080910D013F
:1003C00098E8892780930D0103C08AE58093620035
:1003D000912FEEE0F1E002C08D9181939150E0F712
:1003E000612F8EE091E01ED01C5F109362001F9180
:1003F0000895A82FB92F8FEF9FEF41E050EA615089
:1004000070F02D9138E0722F782796958795269574
:1004100070FF02C0842795273A95A9F7F0CF809501
:1004200090950895E6DF8D939D930895CF93CFB770
:10043000CF93809BFECF809B09C0809B07C0809B91
:1004400005C0809B03C0809B01C09EC0DF93C0910C
:100450001A01DD27CF5DDE4F809B02C0DF91EBCF1D
:100460002F930F931F9300B32FEF00FB20F94F93AF
:100470003F9310B34FEF012700FB21F93BE031C060
:100480004E7F012F10B3216028C0102F4D7F2260B6
:10049000000000B329C04B7F2460012F000010B37F
:1004A0002BC010B3477F28602AC04F7E00B3206165
:1004B0002CC04F7D10B320622FC04F7B00B320644F
:1004C00032C0422700B349934FEF0000102710FBC2
:1004D00020F910B31570A9F1297F91F2012700FBD3
:1004E00021F900B3237F89F23150F0F1102710FB7E
:1004F00022F910B3277E79F2012700FB23F92F7C24
:1005000081F200B3102710FB24F92F7971F200C09B
:1005100010B3012700FB25F92F7359F200C000B377
:10052000102710FB26F9223040F200C010B301273B
:1005300000FB27F9243028F64F77206810B300001D
:10054000F9CF3B503195333010E41ABFB8F0C31BDC
:10055000D0400881033C41F10B3431F11981412F26
:100560001F7720911801121731F4093691F10D32DD
:1005700079F0013E69F0222720931F013F914F91AE
:100580001F910F912F91DF91CF91CFBFCF911895F0
:1005900000931F013F914F911F910F912F91DF9178
:1005A000CAB7C6FD46CFF0CF00911F01002331F33B
:1005B00010911D011123A1F53430A2F130931D01DA
:1005C0000093190110911A013BE0311B30931A017D
:1005D00029C000911D0101301CF50AE547FD09C045
:1005E0003091610034FD20C000936100C2E0D1E091
:1005F0001FC03091620034FD17C000936200CDE04F
:10060000D1E016C0052710E002BB1FC0052722C09D
:10061000052727C005272CC0052710E002BB33C0E3
:100620004AE503C042ED01C0432FC4E1D0E032E00F
:1006300011B31560909A02B311BB5F9355E020E8A7
:1006400020FF052702BB279517951C3FD8F620FFF2
:100650000527279502BB17951C3FC0F620FF0527ED
:100660002795179502BB1C3F98F620FF0527279575
:1006700017951C3F02BB70F600C0499120FF05276B
:1006800002BB279517951C3F38F620FF05272795B5
:1006900002BB17951C3F38F520FF052727951795B6
:1006A00002BB1C3F10F520FF0527279517951C3F1F
:1006B00002BBE8F4242F3A9519F60A7F5F9102BB3A
:1006C00000C010911E01C651D04011F010931801C6
:1006D00010E41ABF016011B31A7F402F4A7F02BB9A
:1006E00011BB42BB4BCF0527D3CF0527D8CF05275A
:1006F000DDCFFC018081807651F58181863039F52E
:1007000083818230D9F0823269F0813001F58091A5
:10071000D9009091DA0090931C0180931B01809185
:10072000DB000AC08091D6009091D70090931C0105
:1007300080931B018091D8009927089583E690E06B
:1007400090931C0180931B0182E290E0089580E069
:1007500090E00895FC012EED30E030931C012093D1
:100760001B0180818076803231F58181813081F476
:10077000E091DC00F091DD000088F189E02DC901F5
:100780000995E091DC00F091DD00808199270895C2
:10079000823049F484EE90E090931C0180931B0119
:1007A00081E090E008958A3031F483818093E40001
:1007B00080E090E0089580E090E00895AC0118C0DA
:1007C00020E030E0E0E3F5E7CF010197F1F72F5F9C
:1007D0003F4F24313105C1F720E030E0E0E3F5E799
:1007E000CF010197F1F72F5F3F4F22333105C1F75A
:1007F000415050408FEF4F3F580711F70895CFE514
:10080000D4E0DEBFCDBFB89A87B3897F87BB88B3FA
:10081000866088BBC09880E395E70197F1F786B3BF
:10082000992786709070959587958230910579F01B
:1008300083309105A1F0019731F05FD59093DD00F1
:100840008093DC0021C081E090E0B8DFFCCF93D33F
:100850009093DD008093DC0081E090E014C0ECD048
:10086000FC019093DD008093DC000284F385E02D91
:1008700009958DD1882329F05FD39093DD00809373
:10088000DC0082E090E09ADFE091DC00F091DD0096
:10089000848195819093D7008093D6008281809344
:1008A000D80080859185009731F09093DA0080938D
:1008B000D900868107C08BE491E09093DA008093A1
:1008C000D90052D58093DB008091D80080937C00C2
:1008D00014BA8FEF85BB88EF82BB85E081BB9EEFAA
:1008E0008FEF9150F1F78150E1F711BA85E083BFA6
:1008F0008FE085BD84EC83BDE091DC00F091DD00EC
:100900000284F385E02D099545DC789400E011E040
:10091000FF2401C010E0A89547DC112341F0E091CD
:10092000DC00F091DD000484F585E02D099508B622
:1009300000FE0EC081E088BF8091E400882341F072
:1009400094E09F1518F0F82E01E002C08BEFF80E2E
:1009500008B607FE17C080E888BF0023A9F4E0911D
:10096000DC00F091DD000484F585E02D0995E0912F
:10097000DC00F091DD000684F785E02D09958823E1
:10098000D9F4C8CF002331F28091620084FFC2CF36
:10099000E091DC00F091DD000088F189E02D8EED22
:1009A00090E00995E091DC00F091DD0060818EED32
:1009B00090E0FDDC00E0AECF01E0E6CFAC9A80E352
:1009C0008A95F1F7AC9820E030E090E048E1842F80
:1009D0008A95F1F7AD98990F9B9B9160842F8A952A
:1009E000F1F7AD9A2F5F3F4F2830310581F7909393
:1009F000E60020E030E048E1842F8A95F1F7AD98D9
:100A000096959B9B9068842F8A95F1F7AD9A2F5FFE
:100A10003F4F2830310581F79093E70008951F93E9
:100A20001FB7F894A49AA59AA398AB9AAD9AAC98DC
:100A3000C5DF1FBF1F9108958EE690E090938A0056
:100A40008093890085E890E00895FC01892B09F4E2
:100A500053C02091E6008091E700682F7727CB01F3
:100A6000807F9070803F910521F481E08093E500C4
:100A700002C01092E500422F552740FF03C02FEF20
:100A800030E002C020E830E041FF02C020E030E06A
:100A900042FF03C08FEF90E002C080E890E043FF88
:100AA00002C080E090E0208381839A01220F232FEF
:100AB000221F330B3195CA018074907075E09595B3
:100AC00087957A95E1F7282BCA018072907033E000
:100AD000959587953A95E1F7282B4071507055957B
:100AE0004795242B22838091E500882329F4862FC3
:100AF0008295807F822B82838091E6009091E7002F
:100B00009093E9008093E800089580919700909178
:100B10009800892B39F0109298001092970021E0EC
:100B200030E00BC042E050E068EE70E086EE90E00E
:100B30001ED4282F332727FD3095C9010895FC01C5
:100B4000AC9A80E38A95F1F7AC9820E098E1892F80
:100B50008A95F1F7AD98892F8A95F1F7AD9A2F5FB5
:100B60002830A9F720E098E1892F8A95F1F7AD9810
:100B70008081880F80839B9902C081608083892F48
:100B80008A95F1F7AD9A2F5F283071F70895CF93CA
:100B9000DF93CDB7DEB721970FB6F894DEBF0FBE57
:100BA000CDBFCE010196CBDF20E030E089818F7090
:100BB000813011F421E030E0C90121960FB6F8949C
:100BC000DEBF0FBECDBFDF91CF910895EF92FF92B0
:100BD0000F931F93CF93DF93CDB7DEB721970FB657
:100BE000F894DEBF0FBECDBF33E0E32EF12CE82238
:100BF000F92206E010E0CE010196A1DF8981992754
:100C00008073907024E0959587952A95E1F78E156D
:100C10009F0529F4F092F300E092F20022C088EBE5
:100C20009BE00197F1F720E030E094E040E3AC9ADC
:100C3000892F8A95F1F7AD98AD9A892F8A95F1F7AA
:100C4000AC98842F8A95F1F72F5F3F4F2F313105F4
:100C500071F780E89BEB0197F1F70150104009F024
:100C6000CACF21960FB6F894DEBF0FBECDBFDF917D
:100C7000CF911F910F91FF90EF900895CF93DF9345
:100C8000CDB7DEB721970FB6F894DEBF0FBECDBF4C
:100C9000CE01019654DF8981282F3327C9018F7037
:100CA0009070019779F58091F0009091F100892B77
:100CB00071F5C90146E0969587954A95E1F781302F
:100CC000910571F0823091051CF4892B79F013C0E5
:100CD0008230910541F0039771F480E090E00AC002
:100CE00081E090E007C082E090E070DF8091F20048
:100CF0009091F3006BDFCE01019621DF89818F7027
:100D0000813029F01092F1001092F00057C081E07C
:100D100090E09093F1008093F00089818093F4003B
:100D200080E797E10197F1F780E08A95F1F720E0FD
:100D300030E050E090E2892F8A95F1F7AD98550F99
:100D40009B9B51600000AD9A2F5F3F4F28303105CB
:100D500091F720E030E090E040E2842F8A95F1F7AF
:100D6000AD98990F9B9B91600000AD9A2F5F3F4F0C
:100D70002830310591F7292F2F77452F4F7797FD91
:100D8000219557FD4195332727FD30958091EA0045
:100D90009091EB00820F931F9093EB008093EA00F9
:100DA000242F332727FD30958091EC009091ED00A2
:100DB000820F931F9093ED008093EC0021960FB665
:100DC000F894DEBF0FBECDBFDF91CF910895A49AF6
:100DD000A59AA398AB9AAD9AAC9850DF8091F40095
:100DE000992756E0969587955A95E1F781309105B8
:100DF00071F0823091051CF4892B31F00895823016
:100E0000910549F0039751F480E090E002C081E041
:100E100090E0DCDE089582E090E0D8DE08958091D5
:100E2000AB009091AC00892B39F01092AC0010927D
:100E3000AB0081E090E008959091F4008091F5007E
:100E40009817E1F42091EA003091EB008091F600D0
:100E50009091F7002817390789F440E050E020917D
:100E6000EC003091ED008091F8009091F900281786
:100E7000390711F041E050E0CA01089581E090E0A7
:100E80000895FC01892B09F456C08091EE009091E1
:100E9000EF00892B41F01082118212821092EF0034
:100EA0001092EE000895A091F4008A2F992766E031
:100EB000969587956A95E1F780836091EA00709135
:100EC000EB008FEF6138780714F481E806C06038D2
:100ED000710514F08FE701C0862F4091EC0050910E
:100EE000ED009FEF4138590714F421E806C040385F
:100EF000510514F02FE701C0242F81832283992705
:100F000087FD90959093F7008093F600332727FD97
:100F100030953093F9002093F800A093F500681BFA
:100F2000790B7093EB006093EA00421B530B5093D4
:100F3000ED004093EC00089589E990E090939E00C5
:100F400080939D008BEC90E09093A2008093A10091
:100F500089E990E00895A49AA59AA398AB9AAD9ACE
:100F6000AC9808958091FA009091FB00891B992715
:100F700087FD909508958DED90E09093B200809359
:100F8000B1008EE091E09093B6008093B5008DEAB9
:100F900090E00895FC01892BD1F18091FA00482F4F
:100FA000552740FF03C02FEF30E002C020E830E0BB
:100FB00041FF02C020E030E042FF03C08FEF90E02D
:100FC00002C080E890E043FF02C080E090E0208310
:100FD0008183CA01880F892F881F990B91959A01E7
:100FE0002074307075E0359527957A95E1F7822B5E
:100FF0009A012072307063E0359527956A95E1F784
:10100000822B4071507055954795842B8283809137
:10101000FA008093FB000895AC9A80E38A95F1F77B
:10102000AC9820E030E040E098E1892F8A95F1F714
:10103000AD98440F9B9B4160892F8A95F1F7AD9A3B
:101040002F5F3F4F2830310581F74093FA00089514
:1010500043B366B355279A0120723070F5E0359599
:101060002795FA95E1F7CA0180719070E3E09595B4
:101070008795EA95E1F7282BCA01887090709595BD
:101080008795282BCA0184709070880F991F282B90
:101090004270507083E0440F551F8A95E1F7242B6E
:1010A0006072262B822F99270895FF920F931F932A
:1010B000CF93DF93EC01A89A00E5802F8A95F1F792
:1010C000C7DFF82E8091D300823020F4F8828FEFB2
:1010D000898321C0A898802F8A95F1F7B9DF182F4E
:1010E000A89A802F8A95F1F7A898802F8A95F1F712
:1010F000A89A802F8A95F1F7A898802F8A95F1F702
:10110000A89A802F8A95F1F7A3DFA8980A95F1F79E
:10111000A89AF88219838A83DF91CF911F910F914A
:10112000FF900895EF92FF920F931F93CF93DF9359
:10113000CDB7DEB729970FB6F894DEBF0FBECDBF8F
:10114000CE010196B2DF8091D300823029F5FB8079
:10115000A7E0EA2EFE2489818770F822E9F004E9ED
:1011600011E1C8010197F1F7CE0104969EDF8E814F
:101170008E259C8189238F2179F0C8010197F1F791
:10118000CE01079692DF89858E259F8189238F2145
:1011900019F083E08093D3009981909599838A8197
:1011A00080958A836B8160956B83292F332720FF7D
:1011B00003C040E050E002C040E850E021FF02C020
:1011C0004FEF50E022FF03C080E090E002C080E8D3
:1011D00090E023FF02C08FEF90E08093FC004093EB
:1011E000FD001092FE009091D3009230A8F18A8108
:1011F000482F552744FF03C081E08093FE0024FF61
:1012000005C08091FE0082608093FE0025FF05C02E
:101210008091FE0084608093FE0045FF05C08091B0
:10122000FE0088608093FE00933011F5262F33274F
:1012300022FF05C08091FE0080618093FE0021FFA7
:1012400005C08091FE0080628093FE0020FF10C0E8
:101250008091FE0080640AC024FF03C081E0809377
:10126000FE0025FF05C08091FE0082608093FE0095
:1012700029960FB6F894DEBF0FBECDBFDF91CF9198
:101280001F910F91FF90EF9008951F93CF93DF93DD
:10129000CDB7DEB723970FB6F894DEBF0FBECDBF34
:1012A0001FB7F894B99AC198BD98C59AA09AA89A00
:1012B00084B3817C84BB85B38E6385BBCE010196EC
:1012C000F4DE8A81282F3327C9018C709070892B16
:1012D00019F081E08093D30025FD03C083E0809363
:1012E000D30020DF1FBF23960FB6F894DEBF0FBEDA
:1012F000CDBFDF91CF911F91089580E291E090934F
:10130000C4008093C3008FEB90E00895009741F0F4
:10131000FC01ACEFB0E083E00D9001928150E1F769
:10132000AFEFB0E0ECEFF0E083E001900D92815080
:10133000E1F708958091D1009091D200892B39F086
:101340001092D2001092D10021E030E00BC043E0B7
:1013500050E06FEF70E08CEF90E009D0282F33273A
:1013600027FD3095C901089582E190E00895FB01C1
:10137000DC0104C08D910190801921F4415050404E
:08138000C8F7881B990B0895C2
:10138800FF5A5A09022200010100803209040000B4
:1013980001030000000921010100012200000705E6
:1013A800810308000A03002B000000000000000F62
:1013B80005DE048505250501000300320000001242
:1013C800000000E7063E060F074107010003003151
:1013D80000000012000000AB070C08B207CA0703A0
:1013E800002B00000000000000450992089A0986B9
:0413F80009010002E5
:00000001FF
